:1000000012C0189518951895189518951895189563
:10001000FFC718951895189518951895189518955F
:100020001895189518958FE58DBFC0E4EEE24E2E19
:1000300084E08EBFD4E0F4E05F2EEEEFF3E0A0E6C4
:10004000B0E088278D933197E9F78CE089B980E09B
:1000500080BD88E18AB955D966248FEF81BB8FEFC7
:1000600087BB80E084BB8CE085BB919884E0809363
:10007000AF0084E08093B10081E08093B00081E024
:100080008093B20080E08FBD85E08EBDBB9A87E68D
:1000900085BD789485E086B980EC87B9E4EBF0E023
:1000A00080E477D958E0C895802D6DD931965A955E
:1000B000D1F704C01F1010101010101FE4EDF0E075
:1000C00088E467D958E0C895802D5DD931965A9556
:1000D000D1F704C01F2020202020201FE4EFF0E0F3
:1000E00080E557D958E0C895802D4DD931965A955D
:1000F000D1F704C01F0101010101011FE4E1F1E09A
:1001000088E547D958E0C895802D3DD931965A9554
:10011000D1F704C01F1015151515101FE4E3F1E009
:1001200080E637D958E0C895802D2DD931965A955B
:10013000D1F704C01F2015151515201FE4E5F1E0C7
:1001400088E627D958E0C895802D1DD931965A9553
:10015000D1F704C01F0115151515011FE4E7F1E0E3
:1001600080E717D958E0C895802D0DD931965A955A
:10017000D1F704C00C12120C20202020A298A3EB6F
:10018000B0E09C9197FF04C09A9B0EC09F779C9310
:100190009A990AC089E19F9399272ED99F919A999C
:1001A00003C090689C9301C0B0C194D88CE0F1D892
:1001B0008FE711E09ED8E8E6FCE184D88FEB11E0F0
:1001C00098D8EAE7FCE17ED8BE9AE8ECF0E088E750
:1001D00090E00197C69A00D9C698FED8482F492BBF
:1001E000C1F784EF91E008D9E3E0F0E0A6EAB0E0DF
:1001F000D3DCE3E0F0E0A0E1B0E0CEDC0F3F09F0BB
:1002000003C089E18093A600E1E0F0E0A0EAB0E05D
:10021000C5DCE1E0F0E0A0E1B0E0C0DC0F3F5FEF63
:10022000150709F006C08FEF90E0A0EAB0E08D93CB
:100230009C9300E010E020E030E0A6E8B0E00D93F1
:100240001D932D933C93A298A3EBB0E09C9197FF54
:1002500004C09A990EC09F779C939A9B0AC089E12B
:100260009F939927C9D89F919A9B03C090689C93AC
:1002700001C09BCF8FEB11E03CD8ECE8FCE122D829
:100280000091A6000A3008F002C002E016D80091E2
:10029000A600043681E008F080E08F930091A6006C
:1002A000093080E010F009F081E09F9189238823D4
:1002B00009F402C001E001D8A6E1B4E0E6EAF0E00A
:1002C000F4DBF3D7E0E9FCE1FDD708E0F6D7A6E8D8
:1002D000B0E08FD748EC50E060E070E0A6E8B0E016
:1002E0000D911D912D913C91BEDB14F009F001C0E0
:1002F00001C051C00027A3E3B0E08C9182FB0EF453
:1003000001E040E0041709F004C084E690E074D8EE
:1003100010C00027A3E3B0E08C9183FB0EF401E052
:1003200040E0041709F004C084E690E065D81BC0E3
:10033000A1CF00E010E020E030E0A6E8B0E00D93AF
:100340001D932D933C93A6EAB0E08C918F5F8C9324
:100350000091A6000F3F10F009F001C003C081E03A
:100360008093A60087CF00E010E020E030E0A6E810
:10037000B0E00D931D932D933C938091A600815086
:100380008093A6000091A600013008F003C08FEF13
:100390008093A6006FCFE3E0F0E0A6EAB0E07BE751
:1003A000EADBBE9AE8ECF0E088E790E00197C69AB5
:1003B00013D8C69811D8482F492BC1F784EF91E084
:1003C0001BD88FEB1AE095D7A6E1B4E0E0EAF0E0A5
:1003D0005DDB6BD7E6E9FCE175D7A6E8B0E009D7AD
:1003E00040E951E060E070E0A6E8B0E00D911D91B9
:1003F0002D913C9138DB14F009F001C001C05BC0C5
:100400000027A3E3B0E08C9182FB0EF401E040E012
:10041000041709F004C084E690E0EED710C000276E
:10042000A3E3B0E08C9183FB0EF401E040E00417FD
:1004300009F004C084E690E0DFD720C0C2CF00E01E
:1004400010E020E030E0A6E8B0E00D931D932D937E
:100450003C93A0EAB0E0DCD6A0EAB0E00D911C919C
:100460000F3F51E0150710F009F001C006C081E010
:1004700090E0A0EAB0E08D939C93A3CF00E010E061
:1004800020E030E0A6E8B0E00D931D932D933C935F
:10049000A0EAB0E0C4D6A0EAB0E00D911C91013012
:1004A00050E0150708F006C08FEF91E0A0EAB0E039
:1004B0008D939C9386CFE1E0F0E0A0EAB0E07BE78B
:1004C0005CDB08D7ECE9FCE1FDD6BE9AECE2F1E09A
:1004D00086E990E00197C69A7FD7C6987DD7482FC6
:1004E000492BC1F784E690E087D7BE9AECE2F1E0B1
:1004F00086E990E00197C69A6FD7C6986DD7482FC6
:10050000492BC1F780E991E077D781E080938200A1
:1005100083E080938300DED68CE03BD7ECD6EEEA16
:10052000FCE1D0D6D5D6E0ECFCE1CCD6BE9AE4E630
:10053000F0E086E990E00197C69A4ED7C6984CD76E
:10054000482F492BC1F784E690E056D7BE9AE4E6DF
:10055000F0E088E592E00197C69A3ED7C6983CD76E
:10056000482F492BC1F784E690E046D7BE9AE4E6CF
:10057000F0E088E592E00197C69A2ED7C6982CD76E
:10058000482F492BC1F784E690E036D7BE9AE4E6BF
:10059000F0E086E990E00197C69A1ED7C6981CD76E
:1005A000482F492BC1F78FEB15E0A3D6E2EDFCE114
:1005B00089D688EC90E020D7BE9AE4E6F0E086E9A0
:1005C00090E00197C69A08D7C69806D7482F492BBE
:1005D000C1F784E690E010D7BE9AE4E6F0E086E941
:1005E00090E00197C69AF8D6C698F6D6482F492BC0
:1005F000C1F78FEB16E07DD6E4EDFCE163D688EC25
:1006000090E0FAD6BE9AE4E6F0E086E990E0019741
:10061000C69AE2D6C698E0D6482F492BC1F784E6A1
:1006200090E0EAD6BE9AE4E6F0E088E592E0019731
:10063000C69AD2D6C698D0D6482F492BC1F784E6A1
:1006400090E0DAD6BE9AE4E6F0E086E990E0019721
:10065000C69AC2D6C698C0D6482F492BC1F78FEB91
:1006600017E047D6E6EDFCE12DD68CE291E0C4D64A
:1006700031D6379A80EC806C87B9C8D7A2E7B0E052
:100680008D939C9381EC806C87B9C0D7A4E7B0E0D0
:100690008D939C9385EC806C87B9B8D7A4E6B0E0C5
:1006A0008D939C9384EC806C87B9B0D7A2E6B0E0C0
:1006B0008D939C933798E2E7F0E0D190E080FF249F
:1006C00000270FD8AAE6B0E03DD8E4E7F0E0D190EB
:1006D000E080FF24002705D8AEE6B0E033D8EEE690
:1006E000F0E0E0D7EAE6F0E0D8D7E2D8EDE0F0E0DD
:1006F00096D7AAE7B0E0EE0C000FE794DD92EC92FB
:10070000EEE6F0E0CFD7EAE6F0E0C7D7C2D8EDE0FA
:10071000F0E085D7ACE7B0E0EE0C000FE794DD9297
:10072000EC92ECE7F0E0D190E0808FEFE7FE8827D5
:10073000F82E082FD6D70BD82F933F934F935F9364
:10074000EAE7F0E0D190E0808FEFE7FE8827F82E0F
:10075000082FC7D75F914F913F912F9113D8EDE0AC
:10076000F0E0AEE7B0E0F3D9EEE7F0E096D7E0E5F1
:10077000FCE1F9D801D908F005C0AEE7B0E0E0E54A
:10078000FCE114D9EEE7F0E088D7E4E5FCE1EBD832
:10079000F3D881E008F480E08F93A2E7B0E00D91F8
:1007A0001C91043650E0150780E010F009F081E05C
:1007B0009F918923882309F45DC0C0988BD58FE76A
:1007C00011E097D5E8EDFCE17DD58FEB15E091D5F3
:1007D000EAEEFCE177D5A6E1B4E0AF93BF93EEE794
:1007E000F0E05BD718D611E002E0BF91AF91F3D8EB
:1007F000E6E1F4E0A6E1B4E0A5D957D581E0809325
:100800009200009192000A3010F009F017C0BE9AD1
:10081000E4E6F0E086E990E00197C69ADDD5C69857
:10082000DBD5482F492BC1F782E390E0E5D5A2E95B
:10083000B0E08C918F5F8C9308F4E3CF1ACFEEE792
:10084000F0E02BD7E4E5FCE18ED896D881E008F003
:1008500080E08F93A2E7B0E00D911C91003050E052
:10086000150781E009F080E09F91892B882309F426
:10087000A4CF01C0C09AE1E0F0E0A0E1B0E08ED9E1
:1008800042E050E0B9D6A0EAB0E00D931C93E3E05B
:10089000F0E0A6EAB0E080D9E6EAF0E0D080EE240D
:1008A000FF2400271ED7A7EAB0E04CD7E0EAF0E02B
:1008B000D190E080FF24002714D749D7E8E5FCE178
:1008C00049D860D7EDE0F0E0A2EAB0E040D9E7EA2D
:1008D000F0E09CD9EDE0F0E0A7EAB0E038D9E2EA38
:1008E000F0E0E0D6E7EAF0E0D8D6A2D7EDE0F0E01D
:1008F000ABEAB0E02CD9ECE5FCE135D8EBEAF0E06E
:10090000CCD696D7EDE0F0E0ACE9B0E020D9E8E550
:10091000FCE129D8ECE9F0E0C0D634D7EDE0F0E016
:10092000ACE9B0E014D9ECE9F0E0BCD6E2E7F0E0E5
:10093000D190E080FF240027D4D67AD7EDE0F0E014
:10094000A3E9B0E004D9E3E9F0E0ACD6E3E9F0E0F4
:10095000A4D66ED7EDE0F0E0A3E9B0E0F8D8E0E689
:10096000FCE101D8E3E9F0E098D60CD7EDE0F0E047
:10097000A3E9B0E0ECD8A7E9B0E0E3E9F0E08DD678
:100980004AD584E294EF90934D0080934C00002769
:10099000A3E3B0E08C9182FB0EF401E040E0041789
:1009A00009F038C088E290E027D50027A3E3B0E043
:1009B0008C9182FB0EF401E040E0041709F02AC09C
:1009C000BE9AEDE7F0E088EC90E00197C69A04D576
:1009D000C69802D5482F492BC1F7A3E8B0E08C9107
:1009E0008F5F8C9300918300063009F003C081E093
:1009F000809383008AE090E0AEE8B0E08D939C9312
:100A000085E08EBD89B7846089BF9A9BFECF8EB585
:100A1000887F8EBD00918200013009F003C083E021
:100A200088BB17C0023009F003C085E088BB11C045
:100A3000033009F003C081E888BB0BC0043009F023
:100A400003C081E188BB05C0053009F002C081E226
:100A500088BB00918300013009F002C055D013C05B
:100A6000023009F002C09BD00EC0033009F002C072
:100A7000DED109C0043009F002C0FCD004C005304A
:100A800009F001C05BD2A4E6B0E08D919C91A0E694
:100A9000B0E08D939C93A0E6B0E00D911C9142E0F4
:100AA00050E0E9D3A0E6B0E04D935C93A0E6B0E05F
:100AB0000D911C91093150E0150708F40EC000910A
:100AC000600048E1041BA1E9B0E00C93A1E9B0E0AB
:100AD0000C914FE0049F0C9203C080E08093910042
:100AE000A0E6B0E00D911C91083250E0150708F423
:100AF00003C08FEF80939100A1E9B0E08C9183BD9A
:100B0000AEE8B0E085D3B5CDAEE8B0E00D911C9174
:100B10000A3050E0150708F001C022C08FEB11E049
:100B2000E8D3EAEEFCE1CED3A6E1B4E0AF93BF9305
:100B3000EEE7F0E0B2D56FD411E002E0BF91AF91E3
:100B40004AD7E6E1F4E0A6E1B4E0FCD7AED3E0EFAB
:100B5000FCE1B8D380E090E0AEE8B0E08D939C93E8
:100B600084E08093AF0084E08093B10081E08093C3
:100B7000B00081E08093B2008FE711E0BAD3E4E5E2
:100B8000FCE1F1D6EEE7F0E088D552D6EDE0F0E0FA
:100B900046D5A5E8B0E0DC92C1D292D208958FEBA1
:100BA00011E0A7D3E2EFFCE18DD3AEE8B0E00D9108
:100BB0001C910A3050E0150708F001C03AC08FEBD5
:100BC00015E097D3E3E9F0E068D5E0E6FCE1CBD6A9
:100BD000D3D681E008F080E08F93E3E9F0E05DD5C3
:100BE000ECE5FCE1C0D6C8D681E008F480E09F9136
:100BF0008923882309F40DC001E05FD3E7E9F0E021
:100C000002E0A6E1B4E0A9D750D3E8EFFCE15AD363
:100C10000AC0E7E9F0E003E0A6E1B4E09ED745D3DF
:100C2000E8EFFCE14FD380E090E0AEE8B0E08D93D8
:100C30009C93A2E7B0E00D911C914FE350E01BD3D1
:100C4000A2E7B0E04D935C9384E08093AF0084E032
:100C50008093B10081E08093B00081E08093B20086
:100C60008FE711E046D3809172008093850056D2C1
:100C700027D20895AEE8B0E00D911C910A3050E003
:100C8000150708F001C0A0C0A2E7B0E00D911C91CB
:100C900042E050E0F0D2A6E7B0E04D935C93A4E7C9
:100CA000B0E00D911C9142E050E0E5D2A8E7B0E041
:100CB0004D935C938FE711E01CD3ECEFFCE102D382
:100CC000A6E7B0E00D911C910A3050E0150708F03E
:100CD00009C002E0F2D2A6E1B4E0E6E7F0E0D6D641
:100CE000E4D22AC0A6E7B0E00D911C91093050E093
:100CF000150780E010F009F081E08F93A6E7B0E0DF
:100D00000D911C91043650E0150781E008F080E059
:100D10009F918923882309F409C001E0CED2A6E17E
:100D2000B4E0E6E7F0E0B2D6C0D206C0A6E1B4E097
:100D3000E6E7F0E0ABD6B9D28FEB11E0DAD2E6ED20
:100D4000FCE1C0D2A8E7B0E00D911C910A3050E060
:100D5000150708F009C002E0B0D2A6E1B4E0E8E768
:100D6000F0E094D6A2D22AC0A8E7B0E00D911C9181
:100D7000093050E0150780E010F009F081E08F9312
:100D8000A8E7B0E00D911C91043650E0150781E012
:100D900008F080E09F918923882309F409C001E0CD
:100DA0008CD2A6E1B4E0E8E7F0E070D67ED206C0CF
:100DB000A6E1B4E0E8E7F0E069D677D280E090E021
:100DC000AEE8B0E08D939C93A2E7B0E00D911C914A
:100DD00045E550E050D2A6E7B0E04D935C93A4E720
:100DE000B0E00D911C9145E550E045D2A8E7B0E098
:100DF0004D935C9385E08093B10082E08093B200D4
:100E000084E08093AF0081E08093B0008FE715E02D
:100E100070D2809176008093850080D18FEB15E0B1
:100E200068D2809178008093850078D10895A2E7F8
:100E3000B0E00D911C914FE750E01DD2A6E7B0E065
:100E40004D935C938FE711E054D2E2EFFCE13AD28C
:100E5000AEE8B0E00D911C910A3050E0150708F0A3
:100E600001C056C08FE715E044D2E3E9F0E015D4A5
:100E7000E0E6FCE178D580D581E008F080E08F9352
:100E8000E3E9F0E00AD4ECE5FCE16DD575D581E04D
:100E900008F480E09F918923882309F40DC001E0C4
:100EA0000CD2E7E9F0E002E0A6E1B4E056D6FDD1CD
:100EB000EEEFFCE107D20AC0E7E9F0E003E0A6E1CB
:100EC000B4E04BD6F2D1EEEFFCE1FCD18FEB11E0B8
:100ED00010D2EAEEFCE1F6D1A6E1B4E0AF93BF9305
:100EE000EEE7F0E0DAD397D211E002E0BF91AF91E4
:100EF00072D5E6E1F4E0A6E1B4E024D6D6D1E0EF85
:100F0000FCE1E0D180E090E0AEE8B0E08D939C930E
:100F100085E08093AF0084E08093B10082E080930D
:100F2000B00081E08093B2008FE719E0E2D18091B8
:100F3000760080938500F2D0C3D00895E2E6F0E019
:100F4000D190E080FF240027CCD3A6E6B0E0FAD30E
:100F5000E4E6FCE108D5E6E6F0E09FD313D4EDE04B
:100F6000F0E0A6E6B0E0F3D58FE711E0C2D1E0E013
:100F7000FDE1A8D1A0E6B0E00D911C910A3050E04F
:100F8000150708F002C001E098D1A6E1B4E0E0E660
:100F9000F0E07CD58AD186E0F6D1E4E0FDE192D1A3
:100FA00001E08BD1E6E0FDE18DD1E6E6F0E075D31E
:100FB000ECE5FCE1D8D4E0D408F002C001E07DD13A
:100FC000A6E1B4E0AF93BF93E6E6F0E066D323D2A8
:100FD00011E001E0BF91AF91FED4E6E1F4E0A6E1BB
:100FE000B4E0B0D562D1EAE0FDE16CD18FEB11E065
:100FF00080D1ECE0FDE166D10091600045E0D6D5FE
:10100000A5E8B0E00C938AD088E290E0F5D108958D
:101010000F921F922F923F924F925F927F92AF92C8
:10102000BF920F931F932F933F934F935F936F93B1
:101030007F938F939F93AF93BF93CF93DF93EF9360
:10104000FF938FB78F93BE9AE4E6F0E088EC90E0D0
:101050000197C69AC1D1C698BFD1482F492BC1F775
:10106000A2E8B0E08C918F5F8C93009182000530F4
:1010700010F009F001C003C081E0809382008091EC
:1010800083008150809383008F918FBFFF91EF91F8
:10109000DF91CF91BF91AF919F918F917F916F9190
:1010A0005F914F913F912F911F910F91BF90AF9002
:1010B0007F905F904F903F902F901F900F901895CA
:1010C0008FEB1AE016D1E2E1FDE1FCD08FEB1DE0E1
:1010D00010D100918200013009F004C0E6E1FDE189
:1010E000F1D01BC0023009F004C0ECE1FDE1EAD010
:1010F00014C0033009F004C0E2E2FDE1E3D00DC00A
:10110000043009F004C0E8E2FDE1DCD006C005309F
:1011100009F003C0EEE2FDE1D5D0089581E08093AF
:1011200084004091850000918400041710F009F0BC
:1011300027C000918400013009F003C083E023D16F
:1011400018C0083009F005C0AFEAB0E08C911BD19F
:1011500010C00C3009F005C0A1EBB0E08C9113D1A8
:1011600008C0003109F003C085E00DD102C084E061
:101170000AD1A4E8B0E08C918F5F8C9308F4D1CFB2
:10118000A5E8B0E08C918F5F8C938091850080936F
:10119000840000918400003110F009F027C0009114
:1011A0008400013009F003C080E0EDD018C00830A1
:1011B00009F005C0A0EBB0E08C91E5D010C00C3078
:1011C00009F005C0A2EBB0E08C91DDD008C0003181
:1011D00009F003C082E0D7D002C081E0D4D0A4E8F7
:1011E000B0E08C918F5F8C9308F4D3CF0895F8947E
:1011F000FFCF0D911D912D913C9181E0080F882723
:10120000181F281F381F3C932E931E930E9308958A
:10121000ED91FC91EF5FFF4FFC93EE930895ED91FC
:10122000FC91E150F040FC93EE93089508D0E4D196
:1012300000FC10D0089503D01ED001F8F9CF00248F
:10124000E89457FF02C009D0689400F80BD010F85A
:101250000124089502D009D00895509540954F5F1C
:101260005F4F0895E89417FF0895009510950F5F5C
:101270001F4F68940895352F242FE894452B11F4BF
:1012800068940895512F402F0027112780E1440FC3
:10129000551F001F111F021B130B416018F4020F92
:1012A000131F4E7F8A9599F70895A6E1B4E08D91BA
:1012B000882311F068D0FBCF089580E264D00A95AE
:1012C000E1F7089543D3802D11F05DD0FBCF089551
:1012D00080EC5FC081E05DD011D080E85AC08FE71C
:1012E000213039F08FEB223021F08FE8233009F0E4
:1012F0008FEC810F4EC080E84CD0089583E0992791
:101300007BC08AEF90E078D08F9A8E9A8D9A8C9AD3
:101310008B9A8A9A929885E090E06ED093989798ED
:101320009698959A949A939AEF93FF93E0E6F0E05B
:1013300050D0FF91EF9193985CD0939AEF93FF93E5
:10134000E0E6F0E046D0FF91EF91939852D0939A67
:10135000EF93FF93E0E6F0E03CD0FF91EF9193989C
:1013600048D09498939AEF93FF93E0E6F0E031D061
:10137000FF91EF9193983DD088E20BD08EE009D099
:1013800086E007D00895929A829505D004D031D096
:1013900008959298F9CF859510F4949A01C0949885
:1013A000859510F4959A01C09598859510F4969AB4
:1013B00001C09698859510F4979A01C09798939AD2
:1013C000EF93FF93E0E6F0E004D0FF91EF91939864
:1013D00008953197F1F70895AE2FBF2F11974A2F37
:1013E0004B2BE1F70895689462F80895E89462F849
:1013F000089581E090E000C0EF93FF93EE27E82B83
:10140000E92B31F0E8EEF3E03197F1F70197D1F7EE
:10141000FF91EF9108958DE207FD8D938F2D881F29
:10142000802F881F8F57082F6894F7F8802F87FF29
:1014300015C080958395082F80E38D938EE28D9360
:10144000802F815228F080E38D9399279C930895F3
:1014500044270A95802F09F192D01FC0805230F0A6
:101460009EE49D9381E48D939D93EFCF4427DF927B
:10147000EF92FF920F938FE1801B11F0082F7FD026
:1014800085D09EE29D930F91FF90EF90DF904427CF
:101490000395003209F4D7CF27D03F93EEE1F5E171
:1014A00038E12F2D1E2D0D2DFF24EE24DD244427A1
:1014B000000F111F221F88F42F923F9247D2102C49
:1014C00045D2202C43D2302C41D23197410DD21C31
:1014D000E31CF01C3F902F9001C0339631963A9553
:1014E00039F73F9107D0B3CFDD0CEE1CFF1C0A95F6
:1014F000D9F70895002719E058D08F93802B11F069
:10150000039501C08F911A95B9F7802F882309F4AC
:101510009ACF8F91805D8D930A95D9F796CF00650C
:10152000CD1D80B2E60E40597307A0ACB90350D66A
:10153000DC01286BEE0094357700CA9A3B0065CD3C
:101540001D00B2E60E0059730700ACB90300D6DCEB
:1015500001006BEE0000357700009A3B0000CD1DC6
:101560000000E60E000073070000B9030000DC0174
:101570000000EE000000770000003B000000F69441
:10158000E794D79447950A95D1F7089500270DD091
:101590008F9303958F2D8E298D29842BC1F78F91E1
:1015A000805D8D930A95D9F750CF1F930F93002735
:1015B00010E2440FDD1CEE1CFF1C001F802F9AE080
:1015C000890B10F0082F43951A9599F7802F0F91EA
:1015D0001F9108952093B8003093B9004093BA004A
:1015E0005093BB0008952091B8003091B90040910C
:1015F000BA005091BB0008950F92B801469F800138
:10160000479F100D569F100D0F900895369A3699EA
:10161000FECF369A3699FECF84B195B108953DD06C
:10162000992711278F2D880F80E8F82A802F881F8F
:1016300008F41FEF41F08F57082F07FD04C0003258
:1016400040F08FEF01C08827982FD82EE82EF82E73
:1016500009C08FE1801B082FF694E794D7949795E3
:101660000A95D1F7112351F09095D094E094F0941D
:1016700081E0980F8827D81EE81EF81E0F2DFE2C3B
:10168000ED2CD92E0895D094E094F09491E0D90EE9
:101690009927E91EF91E10950895D190E190F190D7
:1016A0000191089521913191419151910895102F07
:1016B00090E8FF0C001F0927990FF7941078652F09
:1016C00090E8440F551F5927990F479560780038C7
:1016D0000895FF0C90E89027110F9795F794092F24
:1016E0000895102FBD2CDE2CEF2CF02E11234AF480
:1016F000B094D094E094F0949FEFB91AD90AE90A13
:10170000F90A0EE1FF2039F4FE2CED2CDB2CBB2472
:101710000850C2F76BC032F00A95BB0CDD1CEE1C02
:10172000FF1CF9CF01D0D5CFB7FE089590E8B916C8
:1017300011F4D0FE08959FEFD91AE90AF90A09F4C5
:1017400003950895DD92ED92FD920C930895502F2C
:101750002D2D3E2D4F2D612F08952DEC3CEC4CECA2
:101760005DE366270FC099DFF2DFDD24EE2490E809
:10177000F92E0FE307C096DF05C02227332740E28A
:1017800051E46627552351F1002381F190DF71F177
:101790001627005850580894050B18F407FD03C08D
:1017A00025C007FD23C0469537952795F694E79405
:1017B000D79422D0FF202AF0DD0CEE1CFF1C015034
:1017C00073F09D2D969548F0DD203AF4EE202AF432
:1017D00091E0D90E9927E91EF91E7BCF07C09FE73C
:1017E000092FF92A9FEFD92EE92E0895DD24EE2442
:1017F000FF240027112708959F929924AA24BB242F
:1018000088E1D216E306F40628F0D21AE30AF40AB5
:10181000089401C08894991CAA1CBB1CDD0CEE1C0A
:10182000FF1C8A9571F7D92CEA2CFB2C9F90089508
:101830003EDFE1F25038D1F2162700585058089494
:10184000051F12F418F4CBCF08F0D0CF0AD0FF2038
:101850002AF0BB0CDD1CEE1CFF1C3BCF0F5FFBF125
:1018600038CF9F929924AA24BB24992788E1990C08
:10187000AA1CBB1CDD1CEE1CFF1C30F4920EA31E28
:10188000B41ED91EE91EF91E8A9589F79F90089506
:1018900009DF0DDF503829F090E869270CC00AF005
:1018A00045D017CF5FE322273327442701C0FADE54
:1018B000FEDE5038B1F3003899F3902F951B8BF36F
:1018C00012F434D0FACF983118F022273327442766
:1018D000983028F0232F342F44279850F9CF99239C
:1018E00029F04695379527959A95D9F7912F962700
:1018F00042F014D0B0F6F794E794D7940F5F8BF6CC
:101900006ECF10D051F008F4BEDEFF2052F2DD0C95
:10191000EE1CFF1C0150CBF762CF68CFD20EE31E46
:10192000F41E0895D21AE30AF40A0895DF92EF92A2
:10193000FF920F931F93D22EE32EF42E052F162F16
:101940006F915F914F913F912F910895C895319676
:1019500000200895FBDFD02CF9DFE02CF7DFF02C1E
:10196000F5DF002D0895F2DF202DF0DF302DEEDFC2
:10197000402DECDF502D089507FB00680EF40F7723
:1019800057FB50680EF45F7707FD02C057FF05C094
:10199000D216E306F406050708952D153E054F05FA
:1019A0005007089591E005C092E003C094E001C0A3
:1019B00098E0CCDF0D929A95E1F7089599278D91E3
:1019C00093958823E1F7939511968C9311978E91B7
:1019D0009A95D1F70895EA2FFB2F00244C918D9111
:1019E00003948E32E1F711248D9113948823E1F74B
:1019F0001A94101640F41197202F2119239580E393
:101A00008D932A95E9F7113039F59927AE2FBF2F1D
:101A1000A00DB91FA00FB91F8C919C93853308F4BA
:101A200021C031E08E918E32E9F38D3241F0830F87
:101A30008A3319F480E331E001C033278C93AE1769
:101A400089F7332341F0AE2FBF2FB8DF81E34D324A
:101A500009F43196808308958827E00DF81FE00F80
:101A6000F81F808308950417150726073707089580
:101A7000000F111F221F331F089500951095209508
:101A800030950F5F1F4F2F4F3F4F089501911081E9
:101A90000EC001911191219130810BC001911081F3
:101AA00017FF05C03FEF2FEF04C000811127222749
:101AB000332737FF03C0E1DF8DE28D93CF93DF93B0
:101AC000CF92DF92EF92AA24BB24CC24DD24EE2413
:101AD00040E2CAE0DD2755E093E38881890F87FD66
:101AE0009F7083FD907F891B89935A95A9F7C0DF6A
:101AF000AA1CBB1CCC1CDD1CEE1C4A9551F7E894BB
:101B0000EFE0FF2782910ED0EB30E0F71EF06894F3
:101B10008A2D0CD088278D93EF90DF90CF90DF91A6
:101B2000CF910895982F829501D0892F8F70805D75
:101B300026F0803309F4089568948D9308958827DA
:101B40008D93089581918D938823E1F7089594E012
:101B500081918D939A95E1F7089581918D930A95DE
:101B600019F08823D1F70895EACFE199FECFEEBBB3
:101B7000FFBB3196089591E001C092E07B3751F4AC
:101B80007FB7F894F2DF8D918DBBE29AE19A9A9536
:101B9000C9F77FBF7727089591E001C092E0E5DFA4
:101BA000E09A8DB38D939A95D1F70895FF93881B92
:101BB000F9E0001FFA9511F4FF910895881F841B26
:101BC00018F4840F8894F5CF0894F3CF0FB6F894E7
:101BD0004A925A92E42DF52DA42DB52D480E882752
:101BE000581E0FBE08950FB6F894599049900FBE35
:101BF000089553DD802FFF0C001F901728F4091B58
:101C0000881F0795F7940895F1CDF0CD46DD0023A8
:101C1000E2F3D9F388E0DADF95DD1196FF0C001FBF
:101C20008FE7080F0795F7940695F79483E08F9355
:101C30008EDD88DD139731DDA5DD34DD389738DEA4
:101C400091E0D8DF8F918A9511F08F93F1CFCBCFB0
:101C5000000000000000804000C07F4400002041E0
:101C60000000C8426666A04143414C206C696D6922
:101C70007420706F7765723A00002052656C656160
:101C80007365206B6579212E2E2E0000503D0000DB
:101C900057202F2000002064697600005361766988
:101CA0006E6720706F7765722E2E2E2E00005357B0
:101CB000522F5057522056657220352E3137000072
:101CC00020594F3620202020323031302852292010
:101CD00000005000490052002053575220544F201A
:101CE0004D5554434820212000005357523A0000DC
:101CF00020005057523A000057200000440057007F
:101D000054633D00430055613D00560046414E205E
:101D1000000028423A0038306D29000034306D2927
:101D2000000032306D29000031356D29000031305E
:101D30006D290000FFFFFFFFFFFFFFFFFFFFFFFF19
:00000001FF
